:020000040000FA
:030000000200E11A
:03003300020E9723
:03004B00020BB3F2
:03006B00020F3150
:1000830002082600000080FB1200F0B90003020002
:10009300DBE479127807B800028004F709D8FCE49E
:1000A30090F100785579048002F0A3D8FCD9FA9036
:1000B300F454AA82AB839000F3782979018015E484
:1000C30093A3AC82AD838A828B83F0A3AA82AB8392
:1000D3008C828D83D8E9D9E712227E12008675D0EF
:1000E300007581BF7510007511F102008B79012233
:1000F300FFFFFFFF050D151D252D353D454D555DB5
:10010300656D757DFF0000001B01BE01BE01BE01D0
:10011300BE01C60100E1000012010002020000203E
:100123005104A6160900010203010902430002015A
:1001330000801909040000010202010005240010D7
:10014300010424020205240600010524010001071D
:1001530005820340004009040100020A0000000771
:10016300058402400001070504024000010403095D
:1001730004240354006500780061007300200049E3
:10018300006E0073007400720075006D0065006EF0
:1001930000740073001E034300430031003100313B
:1001A300003100200055005300420020004300446A
:1001B30000430008033000300031003601000059CD
:1001C300010000BB0102E722C082C08389828A83C7
:1001D300BB0003E08002E493D083D08222BB000EF5
:1001E300C082C0838A838982F0D083D08222BB01FC
:1001F30001F722E0F608A3E0F608A3E0F608A3E07F
:10020300F622E6F008A3E6F008A3E6F008A3E6F07A
:1002130022CAC0E0E6F0A308DAFAD0E0FA22CAC0A4
:10022300E0E0A3C582CCC582C583CDC583F0A3C559
:1002330082CCC582C583CDC583DAE6D0E0CA22C3AA
:10024300E498F8E499F91202838026C3E49AFAE465
:100253009BFBE920E7E9120283E498F8E499F92289
:10026300C3E498F8E499F9120283E498F8E499F95D
:10027300C3E49AFAE49BFB22EB20E7CFE920E7E013
:10028300B90010BB0008E88AF084F8AAF022E4FB66
:10029300C8FA22EB70227B10C833C8C933C9335064
:1002A30007C39AC3DBF280069A50012ADBEAC833FC
:1002B300F4C8C933F4C9FA2275F008E4C833C8C9CD
:1002C30033C933C99AC99B5004C92AC93BD5F0EC39
:1002D300FBC833F4C8E4C9FA22600C08C6C313C6CA
:1002E30018C613C6D5E0F422700422600D18C6C3E5
:1002F30033C608C633C6D5E0F41822251010AF085C
:10030300F510400215118008F51040021511D2AF07
:1003130022C0D0251010AF08F51050020511800837
:10032300F51050020511D2AFD0D0222510F582105E
:10033300AF08F510400215118008F51040021511A1
:10034300D2AF851183222510F582E43511F583227E
:10035300E4732510C582C0E0E51134FFC583C0E016
:10036300E510C3958224F9F8E4C5A8858311858235
:1003730010C5A8E8CEF0A3E520F0A37808E608F0BE
:10038300A3DEFAEFF0A3E58124FBF8E608F0A3E689
:1003930008F0A30808E608F0A3E608F0A315811502
:1003A30081D0E0FED0E0F815811581E8C0E0EEC011
:1003B300E022851183851082E0A3FEE0A3F5207877
:1003C30008E0A3F608DFFAE0A3FFE0A3C0E0E0A3A0
:1003D300C0E0E0A3C0E0E0A3C0E0E4C5A8858210CC
:1003E300858311C5A8D083D08222C0D02510C582B1
:1003F300C0E0E51134FFC583C0E0E510C395822456
:10040300F310AF08858311858210800885831185D9
:100413008210D2AFC8F0A3E9F0A3EAF0A3EBF0A3F4
:100423007908E709F0A3D8FAECF0A3EDF0A3EEF016
:10043300A3EFF0A3D0E0F0A3D0E0F0A3D0E0F0A3CB
:10044300E520F0A3E5F0F0A322851183851082E077
:10045300C0E0A3E0F9A3E0FAA3E0FBA37808E0F689
:1004630008A3DFFAE0FCA3E0FDA3E0FEA3E0FFA303
:10047300E0C0E0A3E0C0E0A3E0F5D0A3E0F520A353
:10048300E0A3F5F0E4C5A8858311858210C5A8D043
:1004930082D083D0E0F8D0E0327403800474028009
:1004A30000C0E0F40412032ED0E0120214227403FD
:1004B3008000CCC0E0EDC0E0E510C39CCCAD115092
:1004C300011D10AF068C108D1180068C108D11D27A
:1004D300AF120221D0E0FDD0E0FC22D083D082C550
:1004E300F0E493A3C5F0C395F0F5F0E493A3C395AB
:1004F300F04005E5F0048001E475F002A42582F5DF
:1005030082E5F03583F583E493A3C0E0E493C0E090
:1005130022D083D082E9C0E0E493A3C386F0C5F080
:1005230095F0F908E493A386F0C5F095F0700BE419
:1005330093A3C3994005E9048002A3E475F002A4E0
:100543002582F582E5F03583F583D0E0F9E493A3C2
:10055300C0E0E493C0E022D083D082CCC0E0E49337
:10056300A360061205841470FAE493A360061205CF
:10057300A31470FAD0E0FCE493A3C0E0E493C0E0DA
:1005830022C0E0E493A3D39C5010E493A3C39C4004
:100593000AD0E0D0E0D0E0020577A3A3A3D0E02205
:1005A300C0E0E493A36C7009D0E0D0E0D0E0020592
:1005B30077A3A3D0E02253CBEFC2D843CB0475F08B
:1005C3000CEAA4F5CD74FC55CB4402F5CB43CB1018
:1005D300A2D850FC53CBEFC2D82274F7120355753F
:1005E300084075090078081204A012097112031457
:1005F30090DF36E054EF64016004C2AF80FE90DF09
:1006030037E0C394035004C2AF80FE53BEFBE5BE84
:10061300A2E650FA53C6BF43BE0474F1F5D575D4B0
:1006230045743C90DF13F0741490DF14F0743D9024
:10063300DF02F0740590DF04F0748E90DF2EF07407
:100643000990DF25F0741290DF07F0E490DF08F0E3
:10065300742590DF09F0749590DF0AF0745590DFEC
:100663000BF0741D90DF0CF0745590DF0DF07413D4
:1006730090DF0EF0742390DF0FF0741190DF10F011
:10068300746390DF11F0741D90DF15F0741C90DF1C
:1006930016F074C790DF17F0E490DF18F074B09091
:1006A300DF19F074B690DF1AF0741090DF1BF012AC
:1006B30009D3741F90DF1FF0748890DF23F0743127
:1006C30090DF24F0740290F100F07900120B1E7E8B
:1006D300007F0075E10275081475090590DF3CE0A1
:1006E3005450701F7A407B00120A93E50824C0F52A
:1006F30008E50934FFF509C3E5089401E509120883
:100703001E50D97A10EEC333FEEF33FF90DF3AE089
:10071300A2E0E492E04EFE1AEA70EA74804EF5BC61
:10072300EFF5BC120A5E90F141741412226190F14C
:100733004374FA122261439A01D2AF0210A774F6EE
:10074300120355EAFEEBFF890975080090F100E0FA
:1007530064017004C2AF80FE120A5EEF90F145F0AF
:10076300EE90F146F074DF90F147F074D990F148C0
:10077300F07420120A30744190F14CF0E5097011C5
:1007830043D60175E103E5E9A2E450FA53E9EF80AA
:1007930077740165096004C2AF80FE750A04801B8B
:1007A300120A5E43B404740F55BC04FE90F1431265
:1007B3002435120A931EEE70F3150A43D60175E130
:1007C3000290DF3BE0640D70F87E147F0590DF3C00
:1007D300E0545070197A407B00120A93EE24C0FE55
:1007E300EF34FFFFC3EE9401EF12081E50DF75E1F3
:1007F3000390DF3BE0640D6008E5E9A2E450FA8072
:100803008BE50A709B750801120A5E90F100E064A3
:100813000370031209E5A90802142E9400A2D265FD
:10082300D03322C0E074F11203ED90F100E06403D1
:100833006004C2AF80FEE5E9A2E4502BE5E9A2E63D
:10084300502553E9EF53E9BF539BFCE59B120A5E26
:1008530075083E75090078081204A0120971120385
:10086300141209E502096C53E9EF539BFCE59B75F0
:10087300080275090078081204A090F101E004242D
:1008830001FCE434F1FD7A3F7BF1122789740212F3
:100893000314E0FA90F140E0A2E7400302095B8A07
:1008A3000874012508F8E43400F9E8943FE994005A
:1008B300C365D033400302095BEAC39408500302C3
:1008C300095B90F14DE0704490F13FE0F9120AD5D5
:1008D300E9F090F140E0C2E7F090F1017C5A7DF33A
:1008E300744012022190F364E0FA90F35AE0F87432
:1008F300F828F874FF3400F97402687001E9704D48
:10090300747F6A7048740190F3A3804B7C007B0072
:100913007A008A82A882E82402F582E434F1F5831E
:10092300E0FD121C50E06D70010CE82454F582E4E4
:1009330034F4F583E06D70010B0AEAC3940440D2EA
:1009430074046B608374046C700E0208CB747E6A4B
:100953007006740190F3A2F075083E78081204A0A3
:1009630012097112031443D6017F0202044C7C0066
:100973007D007A017BF112282874022274F8120395
:100983005590F100E064016015E5A8FEC2AFE06494
:10099300037003120A5E7401F0EEA2E792AF7F01C7
:1009A3000203B5C082C083E5C6A2E65004C2AF808D
:1009B300FE90F100E0640170141209D3740290F107
:1009C30000F075E10490DF3BE0640170F8020A8EE9
:1009D30074EA90DF1CF0742A90DF1DF0E490DF1EB0
:1009E300F02274F712035574DF90F145F074D99037
:1009F300F146F074F190F147F0740190F148F0740E
:100A030080120A30741190F14CF075D68175083E4E
:100A130075090078081204A012097112031443D651
:100A230001120A7B75E1024391100210A790F1496C
:100A3300F0744090F14AF0741390F14BF022C082AD
:100A4300C08390F100E064017004C2AF80FEE064F3
:100A53000360067403F01209E58030C082C083533B
:100A630091EF75E10490DF3BE0640170F875D68186
:100A730053D1FE120A7B8013539BFCE59B53E9EF92
:100A830022C082C083740490F33EF0D083D08222CC
:100A930074F71203558A088B09740478081202DC70
:100AA300AE08AF09EA7001EB6025E5A8F508C2AF0F
:100AB3007A107B001205B9E508A2E792AFEEF8EFD2
:100AC300F974FF281E74FF39FFE87001E970DB0237
:100AD30010A7C008C009E9FCC39480401AE9F8795B
:100AE300FF7A027B0012027B8808890974B7250804
:100AF300F874FF3509800CECC313F874B728F87445
:100B0300FF3400F9C3E89480E994FFA2D265D0339F
:100B130050027880E8F9D009D0082274F7120355FF
:100B2300E9FEC394104004C2AF80FE120A5EEE24B5
:100B330058F582E434F4F583E090DF06F090F10099
:100B4300E0640370031209E50210A7E5A8C2AFA28F
:100B5300E7E492E0FA7B0022EAA2E092AF22EBC341
:100B630013FBEA13FAC3EA9402EB94004014000067
:100B73000000000000000000EA24FFFAEB34FFFB52
:100B830080E32274F8120355EAFEEBFFEEF8EFF967
:100B930074FF28FE74FF39FF7400687003740069E2
:100BA30060097AE87B03120B6180E17F010203B5E0
:100BB300C0E074F21203ED90F14EE07002A3E06026
:100BC3000990F14E120FED1203537F0102044C748E
:100BD300F51203558A828B838C088D097E007F0072
:100BE3008008EE250AFEEF3400FFC3EE9508EF956B
:100BF300095011120C0E70EA7A057B00120B861253
:100C03000C0E70DEEEFAEFFB0217B2EEFAE508C344
:100C13009AF9E5822EFCE5833FFD7A137BF2121AE3
:100C2300B7E9F50A22C082C08390F351E0642270D1
:100C33002690F33EE0703F90F3521217E390F2DDFB
:100C43001226A090F2DDE07002A3E06004D291804E
:100C530002C2917402801BE06420701490F33EE0A2
:100C6300701490F34B74D6F0A374F212226180E3F4
:100C7300740490F33EF0020A8EC082C08390F35155
:100C8300E06421701990F33EE0701990F34B74D631
:100C9300F0A374F21213A874071213A18002740450
:100CA30090F33EF0020A8E020A84020A8474F5125B
:100CB30003558A088B098C0A8D0B90F2D67808129B
:100CC3000205E490F2DAF090F2DBF0740890F2DCC3
:100CD300F090F2DDE4F0A31222667A00F9121077A5
:100CE3008A828B83A3A3A3A3A3A3A3E493A2E65023
:100CF3000474018001E490F34AF0E490F349F04373
:100D0300BE80D2BDF512F513F5147515FF7516FFE8
:100D130074FF90DE0BF090DE07F0743E90DE09F076
:100D2300438C10758900C2C5758B00C2E8439A02D3
:100D330053F4FED29043FE01D2AF0217B274F51200
:100D43000355A812E854046020781274FB56F67415
:100D53000290F337F0E490F338F090F33EF0790328
:100D63001213B0751700751800A812E85410600923
:100D7300781274EF56F61210ACA812E8A2E0500FE6
:100D8300781274FE56F6120F51781274FD56F690CF
:100D9300F2DFE07003020E8890F2DDE07002A3E060
:100DA3007003020E88C2AF90DE0E120E8B90DE141B
:100DB300E0A2E0506C90DE16E0FA90DE17E08A0BBA
:100DC30090F210E0F874C0C398F8E49400F98A082C
:100DD300C3E89508E912081E5009E0FA74C0C39AE3
:100DE300FF8002AF0BEF60397508E07509F2750AF1
:100DF30000780812049CEFF97A287BDE1213E8745A
:100E030003120314EFF97CE07DF27A507BF1121A9E
:100E1300B7EF650B700B740490DE0EF0E490DE14F4
:100E2300F090F320E090DE0EF0D2AFC2AF120E8B43
:100E330090DE11E0A2E0404390F2D3E0FE603CC3B9
:100E4300944140027E40EEF97CE07DF27A137BF21E
:100E5300121B1C7508E07509F2750A007808120464
:100E63009CEEF97A287BDE12140C740312031474BB
:100E73000490DE0EF0740190DE11F090F320E09008
:100E8300DE0EF0D2AF0217B2E090F320F0740490BC
:100E9300DE0EF022C0E074F11203EDE5BEA2E650CF
:100EA300FA90DE06E0FAA2E25035A815E890DE0BD0
:100EB300F0F508851609740478081202DCE5089039
:100EC300DE07F0851508851609740978081202DC17
:100ED300E508543E90DE09F090DE01E0D2E0F078C0
:100EE30012EA46F690DE02E0F5087509007404780C
:100EF300081202EB7812E50846F608E50946F69073
:100F0300DE04E0F508750900740978081202EB782D
:100F13001208E50946F6EAA2E050037514017406C7
:100F23005A6003751400758B00C2E802096CC0E0B7
:100F330074F21203EDE5BEA2E650FAE589A2E7508A
:100F430005C2BD120FFA758900C2C5020BCDC0825E
:100F5300C083C29190F331E07002A3E0600990F383
:100F630031120FED120353745390F321F074BE90BA
:100F7300F322F074FC90F323F0744390F324F074A1
:100F8300BE90F325F0740190F326F0747590F32767
:100F9300F0748790F328F0740190F329F074E590CE
:100FA300F32AF0741490F32BF0747090F32CF07414
:100FB300F390F32DF0742290F32EF0758900C2C5DF
:100FC300D2BD90F32F7421F0A374F3F0758221F551
:100FD3008312035390F333E07002A3E0600990F3AC
:100FE30033120FED120353020A8E120FF122E0F8AF
:100FF300A3E0F583888222C082C083E490F326F0C5
:1010030090F327F090F328F090F329020A8DC08221
:10101300C083E9FCEAFD7A007B00800790F336E0A9
:1010230012106190F3351217E390F46EE0687003C9
:10103300A3E069601A1210556C700B90F3351224FB
:101043003512106180091210556D70D0ED60CD021C
:101053000A8E90F336E0F5838882A3E49322F58326
:101063008882E493F890F3351226B390F335E8F0D1
:10107300A3E9F02274F7120355E9FEEAFF1217E918
:10108300800E8A828B83A3A3A3A3A3E4936E60142D
:101093007A007902121011EA7001EB6007EE70E238
:1010A300EF1F70EC7F020203B574F512035590DE57
:1010B3000EE0FEE4F090DE11E0FFA2E4501F748026
:1010C300F0740790F33EF0E5177002E518600985A8
:1010D3001782851883120353E490F33EF0EFA2E2E4
:1010E300500CE490DE11F090F33EF002117590F392
:1010F3003EE06402706590DE16E0F50A90F34B1251
:1011030004B1A90A7A207BDE1213E87403120314D4
:10111300850A081226E912242FE9250A1213909052
:10112300F34EE07002A3E0600474408002744890C0
:10113300DE11F090F34EE07002A3E07016E5177035
:1011430002E5186009851782851883120353E4901A
:10115300F33EF0EE90DE0EF00217B2E06406700983
:1011630085178285188312035390F33EE0600302D0
:1011730012A7EFA2E050DC7508507509F3750A0059
:10118300780812049C79087A207BDE1213E8740332
:1011930012031475170075180090F350E054E01211
:1011A300055A000600BB11202C13401A13804B1262
:1011B300A03813C023132F1290F351E012055A00E5
:1011C3000501371203271205D5110941120B4612E7
:1011D3002F1290F354E07002A3E0705090F356E0A6
:1011E3007002A3E0704690F352E05480F8A3E0F954
:1011F300E87001E9703690F352E090DE00F090F36E
:10120300376018E0640270037403F090F33EE06407
:101213000460030212A174600212A3E0640370EB82
:10122300740280E6790112153AE970DF740490F3D1
:101233003EF080E2790012153AE970CF80EE121980
:101243006180C8121A0B80C390F351E012055A0053
:1012530004006212066712086C120ACE122F1212D1
:10126300144E80A71215F280A290F352E07002A3ED
:10127300E070B990F354E07002A3E070AF90F356BE
:10128300E064017002A3E070A390F34B7438F0A301
:1012930074F31213A874011213A190F33EF0744077
:1012A30090DE11F090F33EE06401600302137C7F53
:1012B3000290F34EC3E09420A3E094004003021392
:1012C3004490F34EE0F50A7F0A807990F337E064A7
:1012D30004600302122F90F350E064816003021252
:1012E3002F90F352E07002A3E0600302122F90F3F9
:1012F30056E064017002A3E0600302122F90F354DE
:10130300E02439F508A3E034F3F50990F34BE5083D
:10131300F0A3E5090212957517AA75180C02122F8E
:101323007517AD75180C02122F75172875180C1246
:101333000C2802120E75177C75180C120C7C021205
:101343000E750A2090F34B1204B1A90A7A207BDEB2
:1013530012140C7403120314850A0812242FE925AE
:10136300081213901226E9EF90DE11F0E50AC394F8
:10137300204003021156021140E06405600302118C
:1013830056851782851883120353021156F9EA34DE
:1013930000FA90F34BE9F0A3EAF0A3EBF022F0A3F9
:1013A300E4F0740122F0A3E4F090F34E2274F712F8
:1013B30003557A008A08E508243FF582E434F3F5FF
:1013C30083E9F00AEAC3940540EA7A008A08E5084B
:1013D3002444F582E434F3F583E9F00AEAC394057F
:1013E30040EA0210A774F6120355EAFCEBFDE9FE8E
:1013F300740A12034912143E600D8C828D83E0122D
:1014030001E012143370F3802274F6120355EAFCE0
:10141300EBFDE9FE740A12034912143E600D12013A
:10142300C68C828D83F012143370F37F030203B5ED
:10143300E9240109EA3400FA1EEE22E0F508A3E0EC
:10144300F509A3E0A908AA09FBEE2274F7120355D4
:1014530090F352E07002A3E0701790F355E0F9E4C3
:101463007001E9700C90F356E064027002A3E0602F
:10147300047404805390F350E01204DE8002741469
:101483008914D214E21490F354E070E590F34AE027
:10149300600478018002780090F358E8122261908A
:1014A300F349E0600A90F358E04402F0A3E4F090BB
:1014B300F33EE06404601590F34B7458F0A374F3A7
:1014C3001213A874021213A190F33EF00210A79016
:1014D300F337E06404709A90F358E4F0A380CF905C
:1014E300F354E0547FF50890F337E064047082E529
:1014F30008C39406400302147490F354E0548060CC
:1015030016121530F583E0640370047801800278C5
:101513000090F358E88094121526F583E064037075
:10152300EE80E8E5082443F582E434F322E5082459
:101533003EF582E434F32274F7120355E9FA90F38B
:1015430056E07002A3E0701290F337E06404601574
:1015530090F354E07002A3E0600B740490F33EF048
:1015630079010210A790F350E0541F1204DE000229
:101573005D157B1583158D1590F352E064016004AE
:10158300790080DEEA90F34980D590F354E0547FEC
:10159300F50890F352E070E8E508C3940650BBE504
:1015A3000890DE0EF090F354E05480601CEA60046F
:1015B30074108002744090DE11F0EA6004740380BA
:1015C30001E4C0E0121530801AEA6004742080023E
:1015D300748090DE14F0EA600474038001E4C0E0D8
:1015E300121526F583D0E0F0E490DE0E0215627446
:1015F300F512035590F353E01204DE01026C160852
:1016030016221657161217E97A00790112101112D1
:1016130017B71201C690F34EF0A3E4F002177690C9
:10162300F352E0FA79001210771217B7E92402098E
:1016330009EA3400FA1201C6FC1919E0FAE9240395
:10164300090909EA3400FA1201C6F9EC90F34EF0E5
:10165300A3E980C790F352E0FE1217E97A007903F9
:10166300121011EE1E70F580A690F34BE4F0A3F078
:10167300A3F0FA02174A750900740378081202EB03
:1016830090F470E02508FBA3E035098B82F583E431
:1016930093C0E090F353E0F8D0E068600302174989
:1016A3008A08750900740378081202EB1217D3E451
:1016B30093C0E090F352E0F8D0E06860030217496A
:1016C3008A08750900740378081202EB1217CEE436
:1016D30093C0E090F355E0F8D0E06870698A08752C
:1016E3000900740378081202EB1217CEA3E493C027
:1016F300E090F354E0F8D0E068704B8A0875090075
:10170300740378081202EB90F470E02508F8A3E064
:101713003509F988828983A3A3A3A3E493F5087405
:101723000193F50990F34BE508F0A3E509F0A374E1
:1017330080F088828983A3A3A3A3A3A3E493F8746B
:101743000193F912269D0A8A0890F4701217E37523
:1017530083F4758272E0C398F50AA3E099F50B74DC
:1017630003780A1202DCC3E508950AE4950B5003DB
:1017730002167990F34BE0FCA3E0FDA3E0FEEC4DF1
:101783004E70047404802490F33EE064046020905F
:10179300F34E1217E37583F375825612226E5009C6
:1017A30090F3561217E312269D740190F33EF07FD7
:1017B300040203B590F34BEAF0A3EBF0A37480F0BB
:1017C30090F34BE0F9A3E0FA7B80221217D3A32214
:1017D30090F470E02508A3E035098B82F583A322FA
:1017E300E0F8A3E0F92290F46CE0F8A3E0F990F3B9
:1017F30035E8F0A3E9F02274F212035574FE1202E5
:10180300FE851082851183EAF0A3EBF01219516073
:101813002B90F474E0FEA3E08007EE2404FEEF3483
:1018230000FF8E828F83E493F8740193F98510820D
:10183300851183E0687003A3E06970DE750E008094
:1018430049749090DE14F074101219427003750BF2
:1018530040750801750900E50A78081202EB8E82CB
:101863008F83A3A3A39355086006E50BD2E0F50B82
:10187300E50B90DE15F0EA90DE13F0E50A12152869
:10188300F583E4F090DE0EF0050E121951FAE50E21
:10189300C39A40030219387A0079051210118A0895
:1018A3008B09AC08AD09EC7001ED60DCEC2402F5AA
:1018B3000CED3400F50D850C82F583E493540FF59C
:1018C3000A90DE0EF0750B008C828D83A3A3A3A375
:1018D300E4932407F508A3E4933400F5097403782B
:1018E300081202DCAA08850C82850D8393A2E740C7
:1018F30003021844744890DE11F074081219427000
:1019030003750B40750801750900E50A7808120292
:10191300EB8E828F83A3A39355086006E50BD2E079
:10192300F50BE50B90DE12F0EA90DE10F0E50A12FB
:10193300153202188374021203147F070203B5F0F1
:101943008C828D83A3A3A3E49354036401228510A3
:1019530082851183120FF1A3A3A3A3E4932274F648
:1019630012035590F337E06402601F90F354E07064
:1019730002A3E0701590F356E07002A3E0700B90A1
:10198300F353E0F9E47001E96008740490F33EF066
:10199300807390F352E0605F7A00F91210778A083F
:1019A3008B09AE08AF09EE7001EF60DE740490F3AB
:1019B30037F090F352E090F338F0750A008E828F7F
:1019C30083A3A3A3A3E493FAE50AC39A5037850A32
:1019D30008E5082439F582E434F3F583E4F07A006A
:1019E30079041210118A828B83A3A3A3E49370EE6C
:1019F3001217FA050A80C690F338F0740390F33790
:101A0300F0F91213B002142E74F712035590F33742
:101A1300E06404701290F350E06401700A90F3568E
:101A2300E07002A3E06008740490F33EF0805490E9
:101A3300F352E0FE90F354E0FF7A0090F338E0F9BC
:101A43001210777A027904121011EA7001EB60D751
:101A53008A828B83A3A3E4936F70E88A828B83A328
:101A6300A3A3E4936E70DC90F352E0C0E090F354D0
:101A7300E02439F8A3E034F3F988828983D0E0F0D5
:101A83001217FA0210A774F7120355EAFEEBFF12BE
:101A93000B4EEE24C0121AADEE24C1121AADEE2481
:101AA300C2121AAD120B5B0210A7F582EF3400F5D8
:101AB30083E4F02274F3120355EAFEEBFF8C0C8DE2
:101AC3000D8909120B4E121B7AF885090AE50A28BB
:101AD300F8E43400F9E894C0E99400C365D03375A1
:101AE3000800502B801B24C2F8EF3400F9121B6A44
:101AF300E0C0E0121B92D0E0121B867002E4F005F6
:101B030008E508C39509EE40DD121B7B2508F0129A
:101B13000B5BA9087F060203B574F3120355EAFEB3
:101B2300EBFF8C0C8D0D8909120B4E750800801C80
:101B3300EE24C1F8EF3400F9121B92E0C0E0121B4F
:101B43006AD0E0121B867002E4F00508E508C3952D
:101B530009500A121B7AFCE508C39C40D3AC081257
:101B63001B7AC39CF080A885080AE50C250AF58238
:101B7300E50D3400F58322EE24C0F582EF3400F541
:101B830083E022F088828983E004F0E064C0228845
:101B9300828983E0FCEE2CF582EF3400F583227416
:101BA300F8120355E9FE90F331747FF0A37409F042
:101BB30090F33374DBF0A3741DF0740790F39EF07D
:101BC300742090F39FF0EA90F3A0F0EB90F3A1F070
:101BD300740790F39AF0742090F39BF0EC90F39CCD
:101BE300F0ED90F39DF0E490F3A2F090F3A3F09066
:101BF300F3A4F090F3A5F01205DD1209A6EEF91295
:101C03000B1E120A4190F39EE064FF6025E090DF13
:101C130005F07A008A82A882E8249EF582E434F3F0
:101C2300F583E0C0E0121C50D0E0F00AEAC394044C
:101C330040E290F468E064FF7004C2AF80FE740178
:101C430090F14DF0740790DF03F00209A1E82468D6
:101C5300F582E434F4F5832274F31203558A0C8B72
:101C63000D90F3A2E07003021CFE120B4EEAF5097D
:101C730090F35AE024F6F50890F363E090F3A5F0AF
:101C830090F364E0FE85080A750B00780A1204A03D
:101C93007C657DF3AA0CAB0D121DD5120314E490E1
:101CA300F3A2F0747E6E704AE5086046121DC3907D
:101CB300F35AF0750A04780A1204A0121DCD120318
:101CC30014780A1204A07C9E7DF37A5F7BF3121DC5
:101CD300D512031490F3A5E090F363F0747F90F3AF
:101CE30064F0EEFA7B00120B5B79007A5A7BF312F5
:101CF3000741AA097B00120B5B8003750800021BD6
:101D03001574F11203558A0E8B0F89098C0C121D61
:101D1300C3250990F35AF0750A04750B00780A126B
:101D230004A0121DCD120314780A1204A07C9E7D18
:101D3300F37A5F7BF3121DD512031490F3A4E090A2
:101D4300F363F0747E90F364F085090A780A120451
:101D5300A0AC0EAD0F7A657BF3121DD5120314EE02
:101D6300FA7B00120B5B7E00801B75080143B404F1
:101D7300E5BC75F04EA4F8A9F0742028FA744E3926
:101D8300FB120B610EEEC3950C502E79017A5A7B30
:101D9300F3120741E9F50870EB7F1480087A017BA1
:101DA30000120B861F90F3A3E07003EF70EFE06067
:101DB300B9E4F090F3A4E004F0A9087F080203B5A6
:101DC300120B4E8A0AAE0A740A227C9A7DF37A5B5E
:101DD3007BF31227417402221209A6120A4122EA56
:101DE3007001EB53F5FE6004D2A08002C2A043FF52
:101DF3000122EA7001EB53F5F76004D2A38002C21B
:101E0300A343FF0822EA7001EB53F5EF6004D2A469
:101E13008002C2A443FF102274F7120355EC700131
:101E2300ED60027C018A088B097808120514000012
:101E330004861E651E401E451E521E5F1E121E890D
:101E4300804153F3FBECA2E0928243FD04803453C0
:101E5300F3F7ECA2E0928343FD08802753F3EFEC02
:101E6300801A121E8953F3FBA2E0928243FD0453AE
:101E7300F3F7A2E0928343FD0853F3EFA2E09284C9
:101E830043FD100210A753F3FDECA2E0928143FD42
:101E9300022274F8120355EAFE74015EFC7D007A97
:101EA300017B00121E1B74025EFC7D007A027B0024
:101EB300121E1B74045EFC7D007A037B00121E1B42
:101EC30074085EFC7D007A047B00121E1B0209A1CC
:101ED30074F512035590F447E07002A3E070030217
:101EE30021ED7E0190F442E01204DE00049E1FFC0B
:101EF3001E5E1FA81FFF1FB82012227664117005F3
:101F0300EE90F442F0EEF890F4351226AF90F435EB
:101F13001226A08E0890F4471226EC90F447E07046
:101F230002A3E070BD90F210E0F5087003022240B6
:101F330090F449E07002A3E070030222401222549D
:101F430090F44985080AC3E0950AA3E0940040038E
:101F53000221C490F449E0FF0221C6740290F442C6
:101F630012227512055A0006437F1F448A1F498EA9
:101F73001F4C921F4E861F52961FA21F744390F44C
:101F8300418081744E80F7744480F3744980EF7408
:101F93004C80EB90F433EEF0A3E4F0E4021F04E48E
:101FA30090F44180F590F441E012055A000543C2D4
:101FB3001F44F11F49F11F4CF11F4EDE1F9E1F12DC
:101FC3002276F8740F5890F41B12226190F41BE0F0
:101FD300FA7B00121E951226F780C0122276A2E029
:101FE300E492E090F41D12226190F41D80E112222C
:101FF3007690F4431222617403021F0490F441E0CB
:1020030012055A00034413204913204C13209E1F2A
:10201300EE90F44B122275F990F443E0F0A3E049FB
:10202300F090F445E4F0A3F090F443E07002A3E0F1
:102033007003021F9E90F42DE07002A3E060030280
:102043001F9E90F42BEE12226190F443E090F43B38
:10205300F090F444E090F43CF090F441E0644C7070
:1020630029741390F439F0744490F43AF07C047DAD
:10207300007A397BF4120BD28A0874046508700164
:10208300EB602DE490F44BF08026741290F439F059
:1020930090F441E06449700474498002744490F4FC
:1020A3003AF01222437C0579047A397BF4121D0439
:1020B3007404021F0490F447C082C08390F443C0A9
:1020C3008290F4451217E37583F4D0821226BCD0B4
:1020D30083D08212226E500690F447E0800B90F476
:1020E30045E0F890F443E0C398F508E508C3942C61
:1020F300400575082C8007E508700302219B90F4C6
:102103004BE0700302218D90F441E0644C701F8515
:102113000882AE82EEFC7D0090F4351226CF8A0A47
:10212300EE650A7001EB6062E490F44B805B12226F
:1021330043E5E290F42F122261E5E3F990F42FE0F6
:102143001226A17C14A90890F4351226C570081232
:102153002680F0A3E48004E490F44BF0E5E290F4ED
:102163003112226190F431E5E3F9E0FAE9FB90F4EE
:102173002F1217E3EAC398F8EB99F97A037B00125D
:10218300028390F431E8F0A3E9F085080A90F4455E
:10219300E0250A122696AE0890F445C08290F443D7
:1021A3001217E37583F4D08212226E5003021F08C4
:1021B300E490F441F090F442F090F42BF0A3021F6A
:1021C30007AF08EFF97CE67DF37A507BF1121B1C15
:1021D300E9F582A88290F447E02812269690F44904
:1021E300C3E098F0A3E09400804B90F210E0F50870
:1021F300604B122254E508C39441400575094080A1
:1022030003850809A9097CA67DF37A507BF1121B8B
:102213001CE990F44712226190F447E0F87440C33C
:1022230098F8E49400F990F4491226A090F43574D8
:10223300A6F0A374F3122266E490F41AF00217B224
:102243007A017B00121DE290F41F74F4F0A3EEF008
:1022530022E490F2DFF07AE87B03120B6122F0A311
:10226300E4F022F0740190F2DFF022C3E098A3E0DF
:102273009922F090F435120FF1E0227A007B0012DC
:102283001E087A007B00121DE27A007B00121DF506
:102293007A007B00121E9553F4FB53FEFB53F6FBAF
:1022A30053F7BF90F429E4F0A3F090F42BF0A3F0DC
:1022B30090F42DF0A3F090F433F0A3F075E40590BF
:1022C300F441F090F442F090F443F0A3F090F4451D
:1022D300F0A3F090F447F0A3F090F4497440122275
:1022E3006190F44C12268DF0A3F090F450F0A3F01B
:1022F30090F452F0A3F090F41AF0748055C6FA5398
:10230300BEFB53C6BFE5C6A2E640FA8AC6E5C66A67
:1023130070FB43BE0453F4FDC29143FE027A507B2B
:10232300F1121A897A137BF2121A8990F4787808D9
:102333001201F6AA08AB09AC0AAD0B120CB01226B7
:10234300F790F414E4F0A3F090F412F0A380067471
:1023530028F0A37423F0120D40121ED312244990C7
:10236300F41FE07002A3E0601990F41FE0640170B1
:1023730002A3E070077A007B00121DE290F41F12A3
:10238300243B90F421E07002A3E0601990F421E073
:1023930064017002A3E070077A007B00121DF590C0
:1023A300F42112243B90F423E07002A3E060359003
:1023B300F425E07002A3E0702490F423E06401703C
:1023C30002A3E070077A007B00121E0890F4231228
:1023D300243B90F42574E8F0A37403800690F4255D
:1023E300122440F0A29290F4275003022352C3E038
:1023F3009410A3E09427402B90F41DE07002A3E017
:1024030090F41D6005E4F0A380057401F0A3E4F0EB
:1024130090F41D122435121E951226F790F427E42A
:1024230002234E90F4271226A602235890F34BE082
:10243300F9A3E0FAA3E0FB22122440F022E024FFF8
:10244300F0A3E034FF2274F512035590F452E070C8
:1024530002A3E070030225FF75080190F44DE0121A
:1024630004DE000483247324A424D724E7247725DB
:1024730090F43712227964127006740190F44DF0CF
:10248300A80890F4371226AF90F4371226A090F4E0
:10249300521226EC90F452E07002A3E070BA0226C6
:1024A3004C90F43712227912055A000341C8244490
:1024B300BA2449C424D424744490F44CF0740280A4
:1024C300BB744980F4744190F44CF0740290F44D61
:1024D300F0E480A890F43712227990F44E1222612E
:1024E3007403809890F437122279F990F44EE0F057
:1024F300A3E049F090F450E4F0A312268DE07002BB
:10250300A3E07003022483741390F43DF0744490A9
:10251300F43EF090F44EE090F43FF090F44F122626
:10252300D88A0A7404650A7001EB7006740490F487
:102533004DF090F44CE0644960030225F690F42BCF
:10254300E07002A3E060030225F6741290F43DF0FC
:10255300744190F43EF07C0579047A3D7BF4121DBE
:1025630004E9640170030225F690F42D7401F0A3CD
:10257300E402248290F4501217E37583F475824EBB
:102583001226BC7583F475825212226E500690F4A3
:1025930052E0800B90F450E0F890F44EE0C398FEC4
:1025A300EE6033F508FC7D0090F4371226CF90F4EB
:1025B3002DE07002A3E060157C05EEF990F437126C
:1025C30026C56401700790F42DE4F0A3F090F45055
:1025D300E0250812269690F44E1217E37583F475DE
:1025E300825012226E5003022483E490F44CF09044
:1025F300F44DF090F42DE4F0A302248290F3A2E0D2
:102603006047E490F2DFF07A207B03120B617AE6F5
:102613007BF3121C5BE9FE60271226801222617A8B
:1026230001FB121DF590F42174F4F0A37401F0EE94
:1026330090F45212226190F43774E6F0A374F3F02D
:1026430090F4141226A612226690F433E07002A3CB
:10265300E0602790F44DE07021741390F43DF07422
:102663005490F43EF090F431E090F43FF090F43263
:102673001226D890F433E4F0A3F00217B27A017B68
:1026830000121E0890F42374C822F090F44DF090C9
:10269300F44E22F0A3E03400F02290F34EE8F0A3CE
:1026A300E9F022E02401F0A3E03400221226B32251
:1026B300E028F8A3E03400F922E0C398F8A3E099F6
:1026C300F922E0FAA3E0FB121D04E922E0FAA3E0F9
:1026D300FB120BD222E090F440F07C047D007A3DA3
:1026E3007BF4120BD22290F34EC3E09508F0A3E0E3
:1026F3009400F022C082C08390F41DE07002A3E036
:1027030090F418600974DE12273874EB800774EBB9
:1027130012273874DEF0A37425F090F41BE0540FF5
:10272300F990F416E0FCA3E0FD90F418122435129E
:102733001BA2020A8EF0A37425F090F4162274F7FC
:102743001203557409120349E0FEA3E0FFEAF8EB14
:10275300F980188C828D83E088828983F0A3A88214
:10276300A9838C828D83A3AC82AD838E088F097479
:10277300FF25081E74FF3509FFE5087002E509709F
:10278300D27F020203B574F7120355740912034989
:10279300E0F8A3E0F9EAFEEBFF8A088B09C3EA9CA1
:1027A300EB9D405EEC28F582ED39F583C3E5829518
:1027B30008E5839509404BEA28FAEB39FBAC82AD77
:1027C300831228177002E5096041EC24FF1CED34E5
:1027D300FFFDEA24FF1AEB34FFFB8C828D83E08A32
:1027E300828B83F080DB8C828D83E08A828B83F003
:1027F3008C828D83A3AC82AD838A828B83A3AA82CE
:10280300AB831228177002E50970DBEEFAEFFB7F4A
:10281300020203B58808890974FF25081874FF3577
:1028230009F9E5082274F81203557408120349E004
:10283300F8A3E0F98A828B838003ECF0A3E8FEE936
:10284300FF74FF2E1874FF3FF9EE7001EF70EB7FFA
:04285300010203B5C6
:04000005000000E116
:00000001FF
